S02000002E2E5C62696E5C6F70656E626C745F73746D3332663039312E73726563AB
S3150800000000100020D513000827140008291400083A
S3150800001000000000000000000000000000000000D2
S315080000200000000000000000000000002B1400087B
S3150800003000000000000000002D1400082F1400081E
S31508000040331400083514000837140008391400085A
S315080000503B1400083D1400083F140008411400082A
S3150800006043140008451400084714000849140008FA
S315080000704B1400084D1400084F14000851140008CA
S31508000080531400085514000857140008591400089A
S315080000905B1400085D1400085F140008611400086A
S315080000A0631400086514000867140008691400083A
S315080000B06B1400086D1400086F140008711400080A
S315080000C010B5064C2378002B07D1054B002B02D020
S315080000D0044800E000BF0123237010BD3C01002046
S315080000E000000000301F0008084B10B5002B03D095
S315080000F00749084800E000BF07480368002B00D1FD
S3150800010010BD064B002BFBD09847F9E7000000000E
S3150800011040010020301F00083C01002000000000BC
S31508000120164B002B00D1144B9D46402292029A1A78
S31508000130924600218B460F461348144A121A01F0BC
S31508000140BFFD0F4B002B00D098470E4B002B00D05D
S3150800015098470020002104000D000D48002802D011
S315080001600C4800E000BF01F085FD2000290000F0E2
S31508000170A5FD01F069FDC04600000800001000203A
S3150800018000000000000000003C0100204806002096
S31508000190000000000000000010B500F045F88021BE
S315080001A08901034800F046FB431E9841C0B210BDC2
S315080001B00008004810B5642000F006F810BDC046D7
S315080001C010B500F007F810BD014B18807047C046FF
S315080001D05C01002010B501F093F9104B1B6898429A
S315080001E01BD30F4B1B78002B08D101220C4B1A701E
S315080001F020219020C00500F023FB07E00022084BD1
S315080002001A7020219020C00500F01CFB01F078F937
S31508000210044B1B881818014B186010BD58010020A4
S315080002205E0100205C01002010B520219020C00549
S3150800023000F008FB10BDC04610B58024A4040121B7
S31508000240200000F031FC0021200000F02DFC10BD3C
S3150800025010B502000368022083431360136801384F
S31508000260034313605368184207D13B4B0124506877
S31508000270044202D1013B002BF9D153680020DB0769
S3150800028069D58B79012B04D110687F33034313603A
S3150800029003E01368802083431360CB79012B04D1D4
S315080002A010683F330343136003E013684020834319
S315080002B013600B7A012B04D110681F3303431360B4
S315080002C003E013682020834313604B7A012B04D183
S315080002D010680F330343136003E013681020834349
S315080002E013608B7A012B04D110680733034313601C
S315080002F003E01368082083431360CB7A012B04D1EB
S31508000300106803330343136003E013680420834330
S3150800031013608B789C07C878030623430879000482
S315080003200343487900050343098801390B43D36120
S31508000330136801218B4313605368194207D0064B93
S3150800034001205168084202D0013B002BF9D15068C0
S3150800035001235840184010BDFFFFFF0070B5837A8F
S31508000360012214009C403A4B802189005D582A439B
S315080003705A508725AD005959E24311405951037B1C
S31508000380002B16D13249103D4B5913404B51837AF5
S31508000390C5882D04468835434833DB005D50837A8B
S315080003A08188090405882943DB002A4DAC46634445
S315080003B05960037B012B17D125498325AD004B597D
S315080003C023434B51837A05882D04468835434833A1
S315080003D0DB005D50837A81880904C5882943DB00E0
S315080003E01C4DAC4663445960C37A002B06D1184DA0
S315080003F0812189006B5813406B5005E0144D81210B
S3150800040089006B5823436B500389002B05D110498B
S3150800041085239B00CD582A40CA500389012B05D154
S315080004200B49852292008B5823438B50437B012B23
S3150800043005D10749872292008B581C438C500449E2
S31508000440802292008B58012083438B5070BDC04692
S31508000450006400404066004000238371C371037244
S3150800046043728372C3728370C37003330371013B93
S315080004704371013B03807047F0B583685B0152D432
S3150800048083681B0151D483680425DB005DD54EE0E3
S31508000490C022520094469E580A6857054A7A3A433B
S315080004A0324366469A510BE0C0267600B4469E59FA
S315080004B04F68FF003A4332434E7A324366469A51B2
S315080004C08A7A0F2632408A72C22252009E580F2715
S315080004D0BE439E509E588F7A3E439E508E7B320670
S315080004E04E7B36041643CA7A16430F7B3F023E43B9
S315080004F02201821810008930FF300660887C0406C5
S31508000500487C00042043CC7B20430C7C2402010059
S3150800051021438D32FF321160C0214900585801220B
S3150800052002435A5011E0002502E0012500E00225A9
S315080005302C002B01C318C02676009A5901273A4089
S315080005409A510A7A002AA3D0AEE72800F0BDC04621
S31508000550012908D0002902D0022908D00BE08268B8
S315080005600F4B134008E082680E4B134004E0826884
S315080005700D4B134000E00023094A93420DD003D8DF
S315080005800220002B0AD006E0064A0120934205D035
S31508000590054A934202D0002000E00120C0B270470D
S315080005A003000004000300080000031070B50B01E7
S315080005B0C318D82464001C5904252C40147205D18C
S315080005C0B134FF341C59640D146004E0D824640067
S315080005D01C59E4085460D82464001C5902252C4090
S315080005E05472B335FF355C590F26344094725B5903
S315080005F01B0AD3740B01C3181C00B934FF342568D1
S31508000600D57225682D0A157325682D0C557324682F
S31508000610240E9473BD33FF331C68D4731C68240AF4
S3150800062014741C68240C54741B681B0E93740029DC
S3150800063004D1C26820231343C36003E00269202360
S315080006401343036170BDC0460300002903D1C36884
S315080006500320184005E00020012902D11B69033058
S3150800066018407047044B1B691B0604D5024B034A06
S315080006705A60034A5A6070470020024023016745C2
S31508000680AB89EFCD024A116980230B43136170478A
S3150800069000200240014BD8607047C0460020024047
S315080006A0084BDB680120DB070AD4064BDB68013000
S315080006B0DB0605D4034BD8684007C00F0423181A75
S315080006C07047C0460020024010B50400FFF7E8FF57
S315080006D0012809D1002C0BD0FFF7E2FF013C0128C5
S315080006E002D1002CF8D103E0002C02D1052000E04D
S315080006F0052010BD70B50500B0200003FFF7E4FF24
S31508000700042810D1084C2369022633432361656106
S315080007102269402313432361B0200003FFF7D4FF67
S315080007202369B343236170BD0020024030B583B00E
S3150800073005000C0000230193B0200003FFF7C4FF57
S31508000740042820D1114A116901230B431361A3B26E
S315080007502B80B0200003FFF7B7FF04280ED102351F
S315080007600195019B240C1C80B0200003FFF7ACFF09
S31508000770064A136901218B43136104E0034A13698E
S3150800078001218B43136103B030BDC04600200240EF
S31508000790F0B54F464646C0B4002500220126032779
S315080007A0330093400C681C40A3423AD10B79013BB5
S315080007B0012B1DD883683C00AC40A3438360846842
S315080007C04B79AB4023438360838898461404230CF3
S315080007D0994633004C46A34044469C43848083880C
S315080007E09C468B794C46A340644623439BB2838040
S315080007F003683C00AC40A343036004680B79AB4034
S3150800080023430360C3689C461404E40B3B00A340DF
S315080008101C006346A343C360C468CB79AB4023433B
S31508000820C36001320235102ABAD10CBC90469946EB
S31508000830F0BDC046008A0840411E8841C0B27047D4
S31508000840816170470185704710B507230B409B00EF
S31508000850C90889004018016A0F249C40A143016217
S31508000860016A9A400A43026210BDC04670B5040088
S31508000870714B5B680C221340042B0CD002D8002B5A
S3150800088005D028E0082B0AD00C2B20D023E06B4B90
S315080008900360002022E0694B036000201EE0664BDF
S315080008A058685A688002000F851CC0235B021A42EA
S315080008B002D16348684308E05F4BDB6A0F211940A1
S315080008C001315E4801F034F96843206006E05D4B6B
S315080008D00360002002E0594B2360002056494B680C
S315080008E01B061B0F584DEB5CDBB226683200DA405C
S315080008F0130062604A685205520FAA5CD2B2D3400E
S31508000900A3600A6BD20502D4504AE26008E04A4A5C
S315080009105268520402D45A08E26001E09A08E2607A
S31508000920454A126B520602D4494A226102E08022E5
S3150800093012022261404A126BD20602D43F4A626111
S3150800094000E066613C4A126B920701D1A36118E088
S31508000950394A126B03210A40012A01D1A66110E027
S31508000960354A126B03210A40022A03D18022120259
S31508000970A26106E0304A126BD243920701D12F4A90
S31508000980A2612D4A116BC0229202114201D1E36184
S3150800099020E0294A116BC02292020A4080214902AE
S315080009A08A4201D1E66115E0234A116BC022920200
S315080009B00A40802189028A4203D180221202E2611A
S315080009C008E01D4A126BC02189020A408A4201D1F9
S315080009D01A4AE261184A116BC0221203114201D168
S315080009E0236220E0144B1A6BC0231B03134080229A
S315080009F0D202934201D1266215E00F4B1A6BC0232F
S31508000A001B03134080221203934203D180231B0247
S31508000A10236208E0084B1B6BC02212031340934263
S31508000A2001D1064B2362044B1B6B1B0602D4054BF4
S31508000A30636200E0606270BD0010024000127A0036
S31508000A4000093D00006CDC02C0000020809FD50034
S31508000A5012800000002904D0044B5A6910435861DB
S31508000A6003E0024A5369834353617047001002400A
S31508000A70002904D0044B9A691043986103E0024A9E
S31508000A80936983439361704700100240002904D09C
S31508000A90044BDA691043D86103E0024AD3698343F9
S31508000AA0D361704700100240002904D0044B1A692C
S31508000AB01043186103E0024A1369834313617047C0
S31508000AC000100240034A136803218B431843106041
S31508000AD07047C04600000140F0B58DB004000D0017
S31508000AE0036801229343036042682B4B13408A68CC
S31508000AF0134343600268294B1A404B68C9680B4385
S31508000B0029690B43134303608268254B13406A69BE
S31508000B101343836002A8FFF7A9FE224B9C4201D12A
S31508000B20089E0AE0204B9C4201D1099E05E01F4B16
S31508000B309C4201D10A9E00E0049E23681B040CD542
S31508000B4076002B6801931900300000F0F1FF0700CA
S31508000B500199300001F072F80AE02B680193190038
S31508000B60300000F0E5FF07000199300001F066F853
S31508000B702A685208002391425B41FF1823681B0428
S31508000B8005D53A07520F0A4B3B401A431700BBB22A
S31508000B90A3810DB0F0BDC046FFCFFFFFF3E9FFFF0D
S31508000BA0FFFCFFFF003801400044004000480040B9
S31508000BB0F0FF0000002904D00268012313430360F4
S31508000BC003E003680122934303607047C905C90D12
S31508000BD001857047808CC005C00D70478268034B3D
S31508000BE0134083608368194381607047FFEFFFFFF6
S31508000BF0C36919400800411E8841C0B27047C04603
S31508000C00264B1A6801210A431A605868244A02408A
S31508000C105A601868234A02401A601868224A024035
S31508000C201A605868214A02405A60DA6A0F208243DD
S31508000C30DA62186B1E4A02401A635A6B8A435A6371
S31508000C4000229A6010311B4A11605A685A605A6825
S31508000C505A605968184A0A405A605A68A021890396
S31508000C600A435A601A68802149040A431A6019001F
S31508000C70802292040B681342FCD0084B5A68032161
S31508000C808A435A60596802220A435A6019000C229C
S31508000C904B681340082BFBD17047C0460010024032
S31508000CA00CB8FFF8FFFFF6FEFFFFFBFFFFFFC0FFD4
S31508000CB0ACFEFFFF00200240FF7FC0FFF0B54746AD
S31508000CC080B482B08027BF0201213800FFF7C2FE38
S31508000CD02023009301266B461E7100249C71032372
S31508000CE098466B4642465A71DC719025ED05694671
S31508000CF02800FFF74DFD20212800FFF7A3FD01215D
S31508000D0080200003FFF7A6FE6B461C71DC7180236A
S31508000D109B01009369462448FFF73AFD01213800F4
S31508000D20FFF7B4FE01213800FFF794FE01220221E5
S31508000D302800FFF789FD012203212800FFF784FD1B
S31508000D400C2300936B4642465A7102271F719C7109
S31508000D50DE7169462800FFF71BFD0121802080040B
S31508000D60FFF794FE01218020C002FFF773FE0F4DA6
S31508000D70042208212800FFF767FD0422092128001C
S31508000D80FFF762FDC0239B0000936B461F71424626
S31508000D905A719C71DE7169462800FFF7F9FC00F06C
S31508000DA0ADFC00F0B9FCFCE7000800480004004868
S31508000DB0F0B55F4656464D464446F0B495B003A88E
S31508000DC0FFF754FD059B01932C4D24239A46AA440C
S31508000DD0233B98462A4B99462A4B9B462E786F7892
S31508000DE0F41901344B465C432100019800F026FFB4
S31508000DF0002909D12100019800F09AFE83B298468D
S31508000E00013B9BB25B4503D90235AA45E6D127E0EB
S31508000E101D48FFF711FA11AC2000FFF71DFB00254E
S31508000E20A571E57125726572A572E572A570E57002
S31508000E30013E2671013F677143462380210012480F
S31508000E40FFF706FA0DA88572C5720123037305809C
S31508000E5045808580C58005814373FFF77FFA06E0E4
S31508000E6093210A4800F01AFC01270126D0E715B09D
S31508000E703CBC90469946A246AB46F0BD141D0008F8
S31508000E8020A10700FF03000000640040EC1C0008D6
S31508000E9030B587B001AB00221A72104C01945A7211
S31508000EA09972002908D0002301AAD218C45CD4720A
S31508000EB00133DAB29142F7D801A90948FFF7DCFAFB
S31508000EC00400074D01E000F0A3FC21002800FFF70D
S31508000ED03FFB0228F7D007B030BDC046E107000047
S31508000EE00064004030B587B0040000211348FFF7BE
S31508000EF0ABFB002300281DD001AD2A0000210F48B6
S31508000F00FFF754FB2A7A0023002A13D10C4A0199C9
S31508000F1091420FD101AB997A00290AD0002301AA80
S31508000F20D218D27AE2540133DAB28A42F7D30123CD
S31508000F3000E00123180007B030BDC0460064004039
S31508000F406706000010B500F041FA10BD70B5551ED1
S31508000F50ADB2002A0AD06D1801350C00461A23785E
S31508000F60335500F055FC0134AC42F8D170BDC0468B
S31508000F7010B500F08FFA00281CD0FFF70DF90028ED
S31508000F8018D000F0FFFB00F0A7FA01210120FFF7B7
S31508000F906FFD00F083FA0100C02280208005FFF76C
S31508000FA0D5FF0320FFF78EFD00F078FA446800F0BD
S31508000FB00FFAA04710BDC04670B506000C4D0024B8
S31508000FC000F026FC2B68B3420BD869688C4663444C
S31508000FD09E4206D263001A199200054B9A18107A97
S31508000FE004E001340C35132CEAD1FF2070BDC0464D
S31508000FF0381D0008F8B54F464646C0B407000068D5
S31508001000FFF7DAFF0023FF2831D0FFF72BFB342048
S31508001010FFF740FBFFF744FB3D1D81239B009946E4
S31508001020B944012803D1FFF72DFB00231FE0042351
S315080010305B42DB1B984643465C193B689C46644406
S315080010402E6800F0E5FB31002000FFF76FFB04284F
S3150800105007D123689E4206D104354D45EBD10124BC
S3150800106002E0002400E00024FFF70CFB2300180030
S315080010700CBC90469946F8BD70B504000D00104B9F
S31508001080984207D00F4B99420AD0FFF7B3FF0028C2
S3150800109001D111E00C4CEB050020002B0FD100E02C
S315080010A0074C2368AB4209D0200020C0802292005A
S315080010B02900FFF74BFF01E0002000E0200070BD8B
S315080010C0600100200020000864030020F0B54F46A8
S315080010D04646C0B483B005000C0016001F004B0A34
S315080010E05B0298460368013306D1434608C080224E
S315080010F092004146FFF72AFF2B68984505D04146DE
S315080011002800FFF7B9FF051E21D02B68E41A2C1911
S315080011100434134B9946434680229200944663440E
S31508001120019300F075FB2B1DE31A4B4506D901996F
S315080011302800FFF7A1FF051E0BD0041D3378237086
S3150800114001340136013F002FEBD1012002E00020D7
S3150800115000E0002003B00CBC90469946F0BDC0469E
S31508001160FF01000001235B42024A1360024A136032
S315080011707047C046640300206001002070B5040073
S315080011800D001600FFF718FF0023FF281BD0681E66
S315080011900019FFF711FFFF2814D0630A5B020B4AF8
S315080011A0934207D12B00320021000948FFF78EFF32
S315080011B0030008E02B00320021000648FFF786FFEF
S315080011C0030000E00023180070BDC0460020000898
S315080011D06001002064030020F0B5474680B404008F
S315080011E00E00FFF7E9FE05000700701E0019FFF75D
S315080011F0E3FE04000020A54271D8043DEDB2FA2DA5
S315080012006DD8162C6BD8FFF72DFA3420FFF742FA63
S31508001210FFF746FA012803D1FFF734FA00205EE00B
S31508001220304B0822904698444646002500F0F0FACE
S315080012303378BB4205D16B005A199200294BD55811
S3150800124004E001350C36132DF0D1143D474600262F
S3150800125000F0DEFA3B78A34205D173009A19920092
S31508001260204BD75805E001360C37132EF0D101274D
S315080012707F42002600F0CCFA43461B78A34206D1EB
S3150800128073009A199200174B9A18526806E00136AD
S315080012900C239C46E044132EECD100227B1B9B18A2
S315080012A0DB0A9BB2002B17D0013B9BB2DB028022E4
S315080012B01201AC181C1900F0ABFA2800FFF71AFA4D
S315080012C0042803D0FFF7DEF9002008E080231B017D
S315080012D09C466544A542EED1FFF7D4F9012004BC2B
S315080012E09046F0BD381D000800B583B0104B1B684A
S315080012F0012001331AD00E4B5A6898688446624416
S315080013001100DA68944661441A69944661445A6938
S31508001310944661449A6994466144DA698B185B423B
S31508001320019301AA04210348FFF728FF03B000BD73
S3150800133060010020C02000080D4B18680D4B1B6883
S31508001340C0180D4B1B68C0180C4B1B68C0180C4BFB
S315080013501B68C0180B4B1B68C0180B4B1B68C018C2
S315080013600A4B1B68C01843425841C0B27047C04672
S315080013700020000804200008082000080C200008A7
S31508001380102000081420000818200008C0200008B3
S3150800139010B50A4B1B68013304D00848FFF72AFE2C
S315080013A000280AD0064B1B680120013305D00448E3
S315080013B0FFF720FE431E9841C0B210BD6001002011
S315080013C064030020004870470020000872B6704782
S315080013D062B6704708498D460849094A094B9B1A5F
S315080013E005DD00240859105104349C42FADB0648EE
S315080013F08047064800470000001000203C1F0008F0
S31508001400C00000203C010020010C00082101000852
S315080014101849194A002301E00B6004319142FBD3B5
S31508001420FFF74CFCFEE7FEE7FEE7FEE7FEE7FEE712
S31508001430FEE7FEE7FEE7FEE7FEE7FEE7FEE7FEE776
S31508001440FEE7FEE7FEE7FEE7FEE7FEE7FEE7FEE766
S31508001450FEE7FEE7FEE7FEE7FEE7FEE7FEE7FEE756
S31508001460FEE7FEE7FEE7FEE7FEE7FEE7FEE7FEE746
S31508001470FEE700003C0100204806002010B5FFF7F3
S3150800148071FE10BD10B5FFF779FE10BD10B5FFF758
S31508001490A3FE10BD10B5FFF74FFF10BD10B5FFF73F
S315080014A091FF10BD10B5FFF71FFF002801D0FFF709
S315080014B06FFF10BD054B00221A60054959609A60F6
S315080014C005211960034B1A607047C04610E000E01A
S315080014D07FBB0000680500200022014B1A60704798
S315080014E010E000E0044B1B68DB0303D5034A1368CE
S315080014F0013313607047C04610E000E0680500201D
S3150800150010B5FFF7EFFF014B186810BD68050020FE
S3150800151010B5040080210A48FFF76AFB002300285B
S315080015200BD0A1B20648FFF751FB054C80212000DD
S31508001530FFF75EFB0028F9D00123180010BDC0464E
S315080015400044004010B5040020210648FFF750FB70
S315080015500023012804D10348FFF73CFB2070012330
S31508001560180010BD0044004010B586B0E1231B02E8
S315080015700093002301930293039305930C3304937A
S31508001580074C69462000FFF7A7FA80214901200089
S31508001590FFF724FB01212000FFF70CFB06B010BD66
S315080015A00044004070B506000C00402903D97F218D
S315080015B0114800F073F82000FFF7AAFF012803D0AE
S315080015C083210D4800F06AF8A3B2002B12D034002C
S315080015D0013B9DB20135751900F01AF92078FFF71D
S315080015E097FF012803D08C21034800F057F80134EF
S315080015F0AC42F1D170BDC0461C1E000870B505008E
S31508001600224B1C78002C13D12148FFF79BFF012899
S315080016103AD11F4B1B78002B33D0FFF771FF1D4BB8
S31508001620186000221C4B1A700132184B1A702BE0F6
S31508001630194B18780130164B1818FFF783FF04006A
S31508001640012812D1144B1A780132D2B21A70104BF3
S315080016501B78934217D192B20D4901312800FFF742
S3150800166075FC0022094B1A700EE0FFF749FF094B7B
S315080016701B6864330024984206D90022034B1A706B
S3150800168002E01C0000E00024200070BDB505002023
S315080016906C050020B0050020B405002010B500F048
S315080016A0B7F8FCE710B500F0ABF8012810D0094BE5
S315080016B01B78012B0CD1FFF723FF074B1B68F5336B
S315080016C0FF33984204D30022024B1A70FFF750FCEE
S315080016D010BDC046B6050020B805002010B5012289
S315080016E0044B1A70FFF70CFF034B1860FFF7DAFF7D
S315080016F010BDC046B6050020B805002010B5FFF796
S3150800170021FC00F081F8FFF7D5FEFFF7B7FE00F0E1
S315080017100DF8FFF7E3FF10BD10B500F079F8FFF7F5
S31508001720E1FE00F013F8FFF7BDFF10BD10B500F09D
S315080017307DF8FFF73DFB044C01232370FFF714FFE8
S315080017400023237010BDC046D000002010B50B48FA
S31508001750FFF7C8FB012805D10122094B1A70074873
S3150800176000F082F80548FFF749FF012805D1002255
S31508001770034B1A70014800F077F810BDBC0500202D
S31508001780D00000207047C04670B505000C00094B14
S315080017901B78012B02D1C9B2FFF77AFB054B1B78E0
S315080017A0002B03D1E1B22800FFF7FCFE00F054F845
S315080017B070BDC046D0000020074B1B78022B05D011
S315080017C0032B05D00820012B05D003E0002002E0FA
S315080017D0002000E040207047D0000020074B1B780F
S315080017E0022B05D0032B05D00820012B05D003E0DA
S315080017F0002002E0002000E040207047D0000020D2
S3150800180010B500F021F810BD10B5FEF7D3FC10BDD9
S3150800181010B5FEF7D5FC10BD034BFE22DA70187121
S315080018200221BA3A99527047FC050020054B00225E
S315080018301A709A6443215A5401315A529A705A704E
S315080018407047C046FC050020024B1878431E984195
S31508001850C0B27047FC05002000214323014AD15439
S315080018607047C046FC05002070B504000378FF2BBE
S315080018701BD1AC4C0023637001252570FF22E27052
S31508001880EF3A22716371FFF797FFA071FFF7A6FF82
S31508001890E071FFF7A3FF000A20726572A57208229D
S315080018A04423E252FFF7EAFD1BE19E4A1278012A19
S315080018B000D036E13733DAB2352A00D90EE1930083
S315080018C0994AD3589F464578FFF776FF01388542EF
S315080018D003DD2220FFF7A0FF03E16278914D281D62
S315080018E0A96CFFF733FBFF23EB706378AA6C944669
S315080018F06344AB64637801334422AB52F1E0457824
S31508001900FFF75AFF0138854203DD2220FFF784FFDF
S31508001910E7E06168834DA9646278281DFFF716FB26
S31508001920FF23EB706378AA6C94466344AB646378D0
S3150800193001334422AB52D4E07A4BFF22DA70426874
S315080019409A64012144229952E5E0764BFF22DA7027
S315080019509A6C4068002808D01018002311785B1884
S31508001960DBB201329042F9D100E000236D4A002033
S31508001970D3710024147254721B0E937201231371CF
S315080019805071907108214333D152C4E0654BFF2250
S31508001990DA70664A9A6400221A715A719A71072196
S315080019A0D9710021197259729972083144229952D3
S315080019B0B1E00020FFF730FF93E05A4BFF22DA70C0
S315080019C000221A71597859719A71DA711A720621B8
S315080019D0443299529FE0534B00221A705A70FF32D4
S315080019E0DA700121BB3A995295E04E4B9D6CFFF790
S315080019F0E3FE621C411E2800FFF744FD002803D1C0
S31508001A003130FFF709FF6CE0464CFF23E370FFF720
S31508001A10D3FE0138A36C9C466044A064012244238B
S31508001A20E25278E04578FFF7C7FE0238854203DDC3
S31508001A302220FFF7F1FE54E03A4BFF22DA7001212B
S31508001A40BB3A99526178002907D1FFF72BFD002888
S31508001A5047D13130FFF7E0FE43E0A21C314B986CCA
S31508001A60FFF710FD002803D13130FFF7D5FE38E027
S31508001A702C4A6378916C8C466344936431E0294C14
S31508001A80FF23E370002525716571FFF795FEA071A8
S31508001A90E5712572657207224423E2523BE04168EC
S31508001AA0204B986CFFF7F2FC002803D13130FFF782
S31508001AB0B3FE16E01B4BFF22DA700121BB3A99529E
S31508001AC029E0FFF755FA174BFF22DA700121BB3AD6
S31508001AD0995220E03120FFF79FFE02E02020FFF711
S31508001AE09BFE43230F4AD35C012B02D11020FFF73C
S31508001AF093FE44230B4AD15E002912DD09480122D0
S31508001B004323C25489B20330FFF73EFE09E044235B
S31508001B10044AD15EF2E74323024AD35C012BF6D18D
S31508001B20E4E770BDFC050020481E0008201F0008D9
S31508001B30002243088B4274D303098B425FD3030AFE
S31508001B408B4244D3030B8B4228D3030C8B420DD311
S31508001B50FF22090212BA030C8B4202D3121209029F
S31508001B6065D0030B8B4219D300E0090AC30B8B42DD
S31508001B7001D3CB03C01A5241830B8B4201D38B038B
S31508001B80C01A5241430B8B4201D34B03C01A524130
S31508001B90030B8B4201D30B03C01A5241C30A8B4273
S31508001BA001D3CB02C01A5241830A8B4201D38B025E
S31508001BB0C01A5241430A8B4201D34B02C01A524102
S31508001BC0030A8B4201D30B02C01A5241CDD2C30974
S31508001BD08B4201D3CB01C01A524183098B4201D3F0
S31508001BE08B01C01A524143098B4201D34B01C01ADB
S31508001BF0524103098B4201D30B01C01A5241C30853
S31508001C008B4201D3CB00C01A524183088B4201D3C1
S31508001C108B00C01A524143088B4201D34B00C01AAD
S31508001C205241411A00D20146524110467047FFE719
S31508001C3001B5002000F006F802BDC0460029F7D01D
S31508001C4076E770477047C046084B10B50400002B6E
S31508001C5002D0002100E000BF054B1868836A002BFC
S31508001C6000D09847200000F033F8C0460000000076
S31508001C702C1F00080E4B70B500251E000D4CE41AEB
S31508001C80A410A54204D0AB00F35898470135F8E7ED
S31508001C9000F020F8084B00251E00084CE41AA41092
S31508001CA0A54204D0AB00F35898470135F8E770BD54
S31508001CB034010020340100203401002038010020BE
S31508001CC003008218934202D019700133FAE770476D
S31508001CD0FEE70000F8B5C046F8BC08BC9E4670474B
S31508001CE0F8B5C046F8BC08BC9E4670472E2E5C2E3A
S31508001CF02E5C2E2E5C2E2E5C536F757263655C41CE
S31508001D00524D434D305F53544D333246305C636118
S31508001D106E2E63000502060206030703080309037D
S31508001D2009040A040B040C040C050D050E050F0521
S31508001D300F0610061007100800200008000800000B
S31508001D400400000000280008000800000500000044
S31508001D5000300008000800000600000000380008EF
S31508001D600008000007000000004000080008000006
S31508001D7008000000004800080008000009000000EC
S31508001D8000500008000800000A000000005800087B
S31508001D90000800000B0000000060000800080000B2
S31508001DA00C00000000680008000800000D00000094
S31508001DB000700008000800000E0000000078000807
S31508001DC0000800000F0000000080000800800000E6
S31508001DD0100000000000010800800000110000004B
S31508001DE000800108008000001200000000000208C0
S31508001DF00080000013000000008002080080000038
S31508001E001400000000000308008000001500000010
S31508001E100080030800800000160000002E2E5C2EAD
S31508001E202E5C2E2E5C2E2E5C536F757263655C419C
S31508001E30524D434D305F53544D333246305C7561D5
S31508001E4072742E6300000000EA190008DC1A000804
S31508001E50DC1A0008D41A0008DC1A0008DC1A000884
S31508001E60C21A0008241A00089E1A00087E1A0008DA
S31508001E70DC1A0008DC1A0008DC1A0008DC1A00085C
S31508001E80DC1A0008DC1A0008DC1A0008DC1A00084C
S31508001E90DC1A0008DC1A0008DC1A0008DC1A00083C
S31508001EA0DC1A0008DC1A0008DC1A0008DC1A00082C
S31508001EB0DC1A0008DC1A0008DC1A0008DC1A00081C
S31508001EC0DC1A0008DC1A0008DC1A0008DC1A00080C
S31508001ED0DC1A0008DC1A0008DC1A0008DC1A0008FC
S31508001EE0DC1A0008DC1A0008DC1A0008DC1A0008EC
S31508001EF04A190008FE180008C6180008381900080C
S31508001F00DC1A0008DC1A0008DC1A00088C1900081C
S31508001F10DC1A0008B2190008BA190008D619000810
S31508001F204F70656E424C540043000000D4000020F8
S30908001F30000000009F
S30D08001F34ECE1FF7F010000004B
S31508001F3C0000000001020304010203040607080955
S31508001F4C0400000000000000000000000000000073
S31508001F5C0000000000000000000000000000000067
S31508001F6C00000000281F0008000000000000000008
S31508001F7C0000000000000000000000000000000047
S31508001F8C0000000000000000000000000000000037
S31508001F9C0000000000000000000000000000000027
S31108001FAC00000000E9000008C100000861
S70508000000F2
